:1000000012C02AC029C028C027C026C025C024C0CD
:1000100023C022C021C020C01FC067C31DC01CC098
:100020001BC01AC019C011241FBECFEDCDBF10E0F8
:10003000A0E6B0E0E6ECF7E002C005900D92A03635
:10004000B107D9F710E0A0E6B0E001C01D92A436D8
:10005000B107E1F724D0B5C3D3CFDF93CF9300D05E
:100060000F92CDB7DEB78B8311C01A82198205C0FB
:1000700089819A8101969A83898389819A812FEF58
:100080008F3F9207A9F78B8181508B838B818823C7
:1000900061F70F900F900F90CF91DF910895DF934C
:1000A000CF93CDB7DEB769970FB6F894DEBF0FBE1A
:1000B000CDBF1C821B82E7E3F0E087E08083A9E5E7
:1000C000B0E0E9E5F0E0808181608C93E2E5F0E06A
:1000D0001082E6E5F0E08FE18083A0E5B0E0E0E5A6
:1000E000F0E0808182608C93A3E5B0E0E3E5F0E08E
:1000F000808182608C9380E88093620080E48093AA
:1001000061001092600084E08A8B85E0898B86E034
:10011000888B1C868C858A878A858D878D858E87BE
:100120008E858F878F858B8B8B898C8B8C898D8B24
:100130008D898093630081E08B8781E0888781E0EF
:100140008F8381E08E8381E08987ECE3F0E080811A
:10015000882F90E0827090700097B9F780E090E06F
:1001600077D28C87ECE3F0E08081882F90E082707A
:1001700090700097B9F781E08D837894E6E3F0E022
:100180008081882F90E088709070009721F48D8195
:10019000813009F0F9C08D81882329F48C858F5F27
:1001A0008C8782E05ADF8C858B3008F01C861D829C
:1001B0008C85282F30E0398F288F888D998D853058
:1001C000910509F487C0288D398D263031051CF53D
:1001D000888D998D8230910509F45FC0288D398D05
:1001E000233031055CF4888D998D0097C9F1288DF5
:1001F000398D2130310509F442C0C6C0888D998DF2
:100200008330910509F451C0288D398D2430310592
:1002100009F453C0B9C0888D998D8830910509F4CF
:1002200086C0288D398D293031056CF4888D998DE3
:100230008630910509F45BC0288D398D2730310552
:1002400009F462C0A1C0888D998D8930910509F4A7
:1002500081C0288D398D2A30310509F48EC094C0B3
:1002600084E08A8B85E0898B86E0888B81E08B87B0
:1002700081E0888781E08F8381E08E8385C01A8A40
:1002800081E0898B82E0888B81E08B8781E08887A1
:1002900081E08F8381E08E8377C01B861C821B8266
:1002A00080E092E09A8389836FC01B861C821B8248
:1002B00080E490E09A83898367C081E08A8B109202
:1002C00061001092600081E08B8781E088871F8247
:1002D0001E825AC081E0898B1092620010926000E9
:1002E00081E08B87188681E08F831E824DC081E07C
:1002F000888B109262001092610081E08B871886D3
:100300001F8281E08E8340C081E08A8B81E0898BEF
:100310008FEF80936200109261001092600081E084
:100320008B8781E0888781E08F831E822DC081E0EA
:10033000898B81E0888B109262008FEF809361003F
:100340001092600081E08B87188681E08F8381E0C6
:100350008E831AC081E08A8B81E0888B8FEF809337
:100360006200109261001092600081E08B8781E052
:1003700088871F8281E08E8307C01B861C821B82B8
:1003800080E190E09A838983E6E3F0E08081882F22
:1003900090E080719070009749F08985813011F468
:1003A000198602C081E0898782E057DEE6E3F0E04B
:1003B0008081882F90E0807290700097D1F0F8943F
:1003C000ECE3F0E08081882F90E0827090700097DD
:1003D000B9F76C8580E090E05FD1ECE3F0E08081DC
:1003E000882F90E0827090700097B9F7789482E03F
:1003F00034DE8C85823039F08C85833021F08C8519
:100400008A3009F08CC08985813009F088C08091DC
:1004100063008F3F49F4809163008F3FE1F38B814C
:100420009C8101969C838B832B813C8189819A815D
:100430002817390709F073C01C821B828A85282F70
:1004400030E03F8B2E8B8E899F8983309105E9F1B7
:100450002E893F89243031057CF48E899F89813033
:10046000910511F12E893F892230310534F58E89AD
:100470009F89009789F04CC02E893F89253031052E
:10048000A9F18E899F898530910544F12E893F8994
:1004900026303105A1F13CC08FEF809362001092AD
:1004A00061001092600034C08FEF809362008FEF84
:1004B00080936100109260002BC0109262008FEF59
:1004C000809361001092600023C0109262008FEF51
:1004D000809361008FEF809360001AC010926200D9
:1004E000109261008FEF8093600012C08FEF8093B5
:1004F0006200109261008FEF8093600009C08FEF5F
:10050000809362008FEF809361008FEF8093600093
:100510008A858F5F8A878A85873008F01A8680915E
:1005200063008F3F09F02ACE8B85813009F026CEFB
:100530008985813009F022CE809163008F3FE1F3FD
:10054000809162008F3F11F481E08D8B809161007A
:100550008F3F11F481E08C8B809160008F3F11F40C
:1005600081E08B8B80916200882309F41D8A809141
:100570006100882309F41C8A80916000882309F4B3
:100580001B8A88858130E1F48D89813059F49A89FC
:100590008F85981739F480916200815080936200B2
:1005A0008FEF8F878D89882359F49A898F859817C3
:1005B00039F4809162008F5F809362008FEF8F87A4
:1005C0008F818130E1F48C89813059F499898E854D
:1005D000981739F4809161008150809361008FEF0A
:1005E0008E878C89882359F499898E85981739F4D8
:1005F000809161008F5F809361008FEF8E878E8185
:100600008130E1F48B89813059F498898D85981770
:1006100039F4809160008150809360008FEF8D8766
:100620008B89882359F498898D85981739F480919E
:1006300060008F5F809360008FEF8D878F858F5F65
:100640008F878E858F5F8E878D858F5F8D8796CD07
:10065000DF93CF9300D0CDB7DEB79A838983ECE3E5
:10066000F0E08081882F90E0827090700097B9F759
:10067000EEE3F0E089819A818083ACE3B0E0ECE3C3
:10068000F0E0808181608C93EDE3F0E080810F9059
:100690000F90CF91DF910895DF93CF9300D00F9209
:1006A000CDB7DEB79A8389836B83ECE3F0E080817A
:1006B000882F90E0827090700097B9F7ECE3F0E03B
:1006C0001082EEE3F0E089819A818083EDE3F0E02F
:1006D0008B8180830FB6F894E29AE19A0FBE0F9057
:1006E0000F900F90CF91DF9108951F920F920FB648
:1006F0000F9211248F939F93AF93BF93EF93FF9328
:10070000DF93CF93CDB7DEB7909163008091620005
:10071000981720F0809162008F3F41F4A8E3B0E089
:10072000E8E3F0E0808181608C9307C0A8E3B0E04B
:10073000E8E3F0E080818E7F8C939091630080915C
:100740006100981720F0809161008F3F41F4A8E389
:10075000B0E0E8E3F0E0808182608C9307C0A8E31A
:10076000B0E0E8E3F0E080818D7F8C9390916300AE
:1007700080916000981720F0809160008F3F41F4D5
:10078000A8E3B0E0E8E3F0E0808184608C9307C0E8
:10079000A8E3B0E0E8E3F0E080818B7F8C93809168
:1007A00063008F5F80936300CF91DF91FF91EF91A2
:1007B000BF91AF919F918F910F900FBE0F901F909F
:0607C0001895F894FFCF2C
:00000001FF
